:10000000B401BB29B416B41EB412B4190B28B4152C
:100010004620031832280830A3005B20A20DA30B52
:100020000D28B41E3D2065206120B41A32203720EF
:1000300022080310B629B416B41EB41234192528A8
:10004000FE39B50034150310B629341A2D28A60040
:10005000341646200318322826084E20031832286A
:10006000B41EB6293D20652034113412B41138086D
:100070008400360884178004432838088400360931
:1000800080058417800544284528B6293720652037
:10009000BA213D2061203508B4190138A20008308A
:1000A000A300A20D03183720031C3D20652061200A
:1000B000A30B512837206520380884003608000536
:1000C000FF3E390884003709402839088400370882
:1000D0003A28A400B5172730A30010307B20033046
:1000E000A300E8307B20A30164307B20A3010A3009
:1000F0007B2024088628A2002508A1002408A0004F
:100100007F212008031DB513B51B0800303EA70052
:100110000711871007108316071187100710F0309A
:10012000860583122708B418B3283A30A100983006
:1001300066213330A600C8201330A1008830662124
:10014000C82064306521C820643065212230A600B3
:10015000C8202830B2200C30B2200630B220B414AF
:100160002708B3283414A600341CC1288710033C88
:10017000031CC628C6200730A100D0306621031416
:1001800008003414FE3C0319B6298714A60E341C4B
:1001900034100715F030860526080F39860407113C
:1001A000A60E3418C828323065210314080004084C
:1001B000A60038088400F030B5050830A700031009
:1001C0000318B50AF120A60CA70BE0280000AB1A13
:1001D000350CF120B9210314F1202F08A3002E08BB
:1001E00059298413AB1F0029000836042B1F36063B
:1001F0008000841700083604031C360680000B2993
:1002000000083604031C36062B1B360680008417B4
:10021000360980050B292B081F39003EA1002A084A
:100220000E3E0318A10A00006629B5132908031918
:10023000B5170530A8002730A30010302B2103305C
:10024000A300E8302B21A30164302B21A3010A3045
:100250002B2124083229A2002508A1002408A0008F
:100260007F212008A000A8030319B513290803194A
:100270003C292802031808002008031DB513B51BEC
:100280000800303EB129A000A00DA00DA00D38300F
:10029000A005813020049F000030A100323066218B
:1002A0001F151F1951291E08A10083161E08B62903
:1002B000A301A200FF30A207031CA307031CB62959
:1002C0000330A100E63066215A29A101FC3EA000BE
:1002D000A109031C7129FF300000A00703186C2935
:1002E000A0076400A10F6B290800013EA7000A3097
:1002F000A200A3017F21A70B7A292408080010304F
:10030000A600A501A401210DA40DA50D2208A4029B
:100310002308031C230FA502031895292208A4070C
:1003200023080318230FA5070310A00DA10DA60B8A
:1003300083292008B6291030A800A101A001A70C2C
:10034000A60C031CA9292208A00723080318230FC1
:10035000A107A10CA00CA50CA40CA80B9F29240894
:10036000B629840031088A00300882008313031301
:100370008312640008008316DF30850084309F00FC
:10038000703086008113870183128A11702BFE3032
:100390008A01872001308A01872050308A01872016
:1003A00061308A0187206C308A0187206D308A0194
:1003B000872020308A0187204C308A0187206930CD
:1003C0008A0187206E308A0187206B308A0187205E
:1003D00020308A01872031308A0187202E308A011F
:1003E000872030308A0187200130A300F4308A0151
:1003F0005921FE308A018720C0308A018720503081
:100400008A01872072308A0187206F308A01872015
:1004100064308A01872075308A01872063308A0121
:10042000872065308A01872064308A018720203048
:100430008A01872062308A01872079308A018720EB
:1004400020308A01872069308A0187207A308A012A
:10045000872075308A01872040308A01872001304B
:10046000A300F4308A015921080000308A01432199
:10047000C0002108C1000A308A01582101308A01D8
:100480004321C4002108C5000A308A015821080010
:100490003E08A6003F08A7000430A200A3018A017D
:1004A0009B21BA002508BB000730B8001030B60009
:1004B0000730B9000830B700A0308A011D203B0882
:1004C0008A011D203A088A011D2041088A011D2049
:1004D00040088A011D2045088A011D2044088A0120
:1004E0001B200A308A01582108003E08A6003F0858
:1004F000A7000430A200A3018A019B21BA002508AD
:10050000BB000730B8001030B6000730B900083023
:10051000B700A0308A011D203B088A011D203A083F
:100520008A011D208A010420C1008A010420C00024
:100530008A010420C5008A010220C4000A308A0111
:10054000582108004008A0004108A10003308A019A
:100550007521C8004008A0004108A10002308A01AE
:100560007521C9004008A0004108A10001308A019E
:100570007521CA004008A0004108A10000308A018E
:100580007521C200C3014408A0004508A100033042
:100590008A017521CB004408A0004508A100023063
:1005A0008A017521CC004408A0004508A100013053
:1005B0008A017521CD004408A0004508A100003043
:1005C0008A017521C600C7010730B8004030B60067
:1005D0005430AA00AB01AE01AF0153308A01D820DC
:1005E0002C308A01D820A9014808A400A501D730E1
:1005F000B000B1018A011521A9014908A400A50193
:10060000D730B000B1018A011521A9014A08A40020
:10061000A501D730B000B1018A011521A901420816
:10062000A4004308A500D730B000B1018A0115210C
:100630002C308A01D820A9014B08A400A501D7308D
:10064000B000B1018A011521A9014C08A400A5013F
:10065000D730B000B1018A011521A9014D08A400CD
:10066000A501D730B000B1018A011521A9014608C2
:10067000A4004708A500D730B000B1018A011521B8
:100680000D308A01D8200A308A01D8200800FE30B7
:100690008A01872001308A01872054308A0187200F
:1006A0004D308A01872050308A0187203D308A01F1
:1006B00087204108A50040088A016920FE308A0190
:1006C0008720C0308A01872056308A0187203D303C
:1006D0008A0187204508A50044088A01692008008E
:1006E0008501860187018A01C7218A0135228A0195
:1006F000A2228A01472346308A0158218A01752B9C
:0607000063008A01802B5A
:02400E00753DFE
:024214000000A8
:00000001FF
